:100000000C944F1F0C94CC1F0C94D51F0C94000023
:100010000C9400000C9400000C9400000C94000060
:100020000C9400000C9400000C9400000C94000050
:100030000C9400000C9400000C9420200C94000000
:100040000C9400000C9400000C94DD1F0C94000034
:100050000C9400000C9400000C9400000C94000020
:100060000C9400000C9400000C9400000C94000010
:100070000C9400000C9400000C9400000C94000000
:100080000C9400000C9400000C940000B600A75AD9
:1000900000B4B50058A700B900000000B800A55989
:1000A00000B4B5005AA900BB00000000B900A45775
:1000B00000B4B5005CAB00BC00000000BA00A35562
:1000C00000B3B4005EAE00BD00000000B900A05453
:1000D00000B3B40061AF00BC00000000B7009D5346
:1000E00000B2B30063B000BA00000000B4009B523D
:1000F00000B0B10065B000B700000000B100985139
:1001000000AFB00067B000B400000000B10098512B
:1001100000AFB00067B000B400000000B2009A5118
:1001200000B1B20065B000B500000000B3009C5201
:1001300000B3B40062AE00B600000000B4009E53ED
:1001400000B5B60060AD00B700000000B500A054D7
:1001500000B6B7005EAC00B800000000B600A255C3
:1001600000B7B8005BAB00B900000000B600A456B1
:1001700000B8B90059A900B900000000B600A657A0
:1001800000B9BA0057A700B900000000B600A7598F
:1001900000B9BA0055A600B900000000B600A95B7E
:1001A00000B8B90054A400B900000000B600AB5D6F
:1001B00000B7B80053A200B900000000B500AC6061
:1001C00000B6B70052A000B800000000B400AD6255
:1001D00000B5B600519E00B700000000B300AE6449
:1001E00000B3B400509C00B600000000B200B0673D
:1001F00000B1B2004F9A00B500000000B100B06934
:1002000000AFB0004F9800B400000000B100B0692A
:1002100000AFB0004F9800B400000000B300B0671A
:1002200000B0B1004F9A00B600000000B500AF6505
:1002300000B1B200519D00B800000000B700AE63ED
:1002400000B2B300529F00BA00000000B800AD61D8
:1002500000B3B40053A100BB00000000B900AC5FC4
:1002600000B4B50054A400BC00000000BA00AB5DAF
:1002700000B4B50056A600BD00000000BB00AA5B9C
:1002800000B4B50058A800BE00000000BB00A85A8A
:1002900000B4B50059AA00BE00000000BA00A6587C
:1002A00000B4B5005BAB00BD00000000B900A4566F
:1002B00000B4B5005DAC00BC00000000B800A15562
:1002C00000B3B4005FAD00BB00000000B7009F5456
:1002D00000B2B30061AE00BA00000000B5009D534B
:1002E00000B1B20063AF00B800000000B3009A5143
:1002F00000B0B10065B000B600000000B100985138
:1003000000AFB00067B000B400000000B100B069F9
:1003100000AFB0004F9800B400000000B400B06718
:1003200000B0B100509B00B700000000B700B065FE
:1003300000B2B300519D00BA00000000B900AF63E5
:1003400000B3B40052A000BC00000000BA00AE60D0
:1003500000B3B40053A300BD00000000B900AB5EC1
:1003600000B4B50055A400BC00000000B800A95CB2
:1003700000B4B50057A500BB00000000B600A75AA6
:1003800000B4B50058A700B900000000B600A75A95
:1003900000B4B50058A700B900000000BA00AA5C7C
:1003A00000B4B50057A600BD00000000BD00AE5E61
:1003B00000B4B50055A600C000000000C000B16048
:1003C00000B3B40053A500C300000000BF00B36336
:1003D00000B3B40052A300C200000000BB00B2652D
:1003E00000B2B300519F00BE00000000B600B2672B
:1003F00000B0B100509B00B900000000B100B0692E
:1004000000AFB0004F9800B400000000B100B06928
:1004100000AFB0004F9800B400000000B200B0661A
:1004200000B2B3004E9A00B500000000B300AE6405
:1004300000B5B6004F9C00B600000000B400AD61EE
:1004400000B8B9004F9E00B700000000B500AC5ED8
:1004500000BABB0050A000B800000000B600AB5BC3
:1004600000BCBD0050A200B900000000B600A959B0
:1004700000BEBF0051A400B900000000B600A7569E
:1004800000C0C10052A600B900000000B600A6548A
:1004900000C0C10054A700B900000000B600A4537A
:1004A00000BEBF0057A900B900000000B600A2526C
:1004B00000BCBD0059AB00B900000000B500A0525F
:1004C00000BABB005CAC00B800000000B4009E5154
:1004D00000B8B9005FAD00B700000000B3009C5148
:1004E00000B5B60062AE00B600000000B2009A503F
:1004F00000B2B30064B000B500000000B100985134
:1005000000AFB00067B000B400000000B100985127
:1005100000AFB00067B000B400000000B4009B5111
:1005200000B0B10065B100B700000000B7009D53F6
:1005300000B1B20063B000BA00000000BA00A054DD
:1005400000B2B30061B000BD00000000BC00A355C4
:1005500000B3B4005FAF00BF00000000BE00A656AD
:1005600000B4B5005DAF00C100000000C000A85895
:1005700000B4B5005BAE00C300000000C200AB5A7F
:1005800000B4B50059AD00C500000000C200AD5B6D
:1005900000B4B50058AB00C500000000C000AE5D5F
:1005A00000B4B50056A800C300000000BE00AF5F55
:1005B00000B4B50054A600C100000000BC00AF614B
:1005C00000B3B40053A300BF00000000BA00B06342
:1005D00000B2B30052A000BD00000000B700B0653B
:1005E00000B1B200519D00BA00000000B400B16734
:1005F00000B0B1004F9B00B700000000B100B0692F
:1006000000AFB0004F9800B400000000B100985156
:1006100000AFB00067B000B400000000B6009B520D
:1006200000B0B10065B200B900000000BB009F53EC
:1006300000B2B30063B200BE00000000BF00A354CC
:1006400000B3B40061B300C200000000C000A555B3
:1006500000B3B4005EB100C300000000BD00A657A7
:1006600000B4B5005CAE00C000000000BA00A6599E
:1006700000B4B5005AAA00BD00000000B600A75A99
:1006800000B4B50058A700B900000000A3C29D64E3
:10069000C6A1A2C4629DC3A600000000A3C3A061BE
:1006A000C5A1A2C5649BC2A600000000A2C3A25EB1
:1006B000C5A0A1C56897C2A500000000A0C4A45CA5
:1006C000C49E9FC66B94C1A3000000009CC5A55AA0
:1006D000C39A9BC76F90C09F0000000098C6A559A1
:1006E000C29697C8748BC09B0000000000000000F9
:1006F00000000000008BC09B000000000000000014
:10070000000000000083B89F00000000000000000F
:1007100000000000007BB0A300000000000000000B
:10072000000000000073A8A5000000000000000009
:1007300000000000006BA0A6000000000000000008
:1007400000000000006398A6000000000000000008
:100750000000000000000000006400000000000035
:100760000000000000000000005000000000000039
:100770000000000000000000004900000000000030
:100780000000000000000000005000000000000019
:1007900000000000000000000064000000000000F5
:1007A0000000000000000000007F000000000000CA
:1007B0000000000000000000009B0000000000009E
:1007C000000000000000000000AF0000000000007A
:1007D000000000000000000000B600000000000063
:1007E000000000000000000000AF0000000000005A
:1007F0000000000000000000009B0000000000005E
:100800000000000000000000008000000000000068
:100810000000000000000000006400000000000074
:100820000000000000000000005000000000000078
:10083000000000000000000000490000000000006F
:100840000000000000000000005000000000000058
:100850000000000000000000006400000000000034
:100860000000000000000000007F00000000000009
:100870000000000000000000009B000000000000DD
:10088000000000000000000000AF000000000000B9
:10089000000000000000000000B6000000000000A2
:1008A000000000000000000000AF00000000000099
:1008B0000000000000000000009B0000000000009D
:1008C00000000000000000000080000000000000A8
:1008D00000000000006398A6000000000000000077
:1008E00000000000006BA0A6000000000000000057
:1008F000000000000073A8A5000000000000000038
:1009000000000000007BB0A3000000000000000019
:10091000000000000083B89F0000000000000000FD
:1009200000000000008BC09B0000000098C6A55C82
:10093000C29697C8748BC09B0000000098C5A55C48
:10094000C39697C7748BC09B000000009CC5A55C34
:10095000C39A9BC76F90C09F00000000A0C4A45D15
:10096000C49E9FC66B94C1A300000000A2C3A25FF7
:10097000C5A0A1C56897C2A500000000A3C3A061DF
:10098000C5A1A2C5649BC2A600000000A3C19D64CE
:10099000C6A1A200629D00A600000000B2C0A55C36
:1009A000C5B0A200629D00A600000000BEBFAA570D
:1009B000C4BCA200629D00A600000000C8BEAF52E9
:1009C000C3C6A200629D00A600000000D1BDB34EC8
:1009D000C2CFA200629D00A600000000DABDB74AA7
:1009E000C2D8A200629D00A600000000DA00B74A4B
:1009F00000D8A200629D00A600000000DA00BA47FD
:100A000000D89D005FA000A100000000DA00BD44F6
:100A100000D899005CA3009D00000000DA00C140EE
:100A200000D894005AA5009800000000DA00C43DE8
:100A300000D88F0057A8009300000000DA00C839E2
:100A400000D88A0054AB008E00000000DA00D031DC
:100A500000D884003EC1008880000000DA00C83958
:100A600000D88A0054AB008E77000000DA00C04145
:100A700000D890006A9500946E000000DA00B84932
:100A800000D89600807F009A65000000DA00B0511F
:100A900000D89C00966900A05C000000DA00A8590C
:100AA00000D8A200AB5400A653000000DE00AE53F5
:100AB00000DC9D00AB5400A100000000DA00A85942
:100AC00000D8A200AB5400A600000000D600A25F30
:100AD00000D4A700AB5400AB00000000D2009C651E
:100AE00000D0AC00AB5400B000000000CE00966B0C
:100AF00000CCB100AB5400B500000000CA009071FA
:100B000000C8B500AB5400B900000000CA009071E5
:100B100000C8B500AB5400B900000000CE00966BD1
:100B200000CCB100AB5400B500000000D2009C65C1
:100B300000D0AC00AB5400B000000000D600A25FB3
:100B400000D4A700AB5400AB00000000DA00A859A5
:100B500000D8A200AB5400A600000000DE00AE5397
:100B600000DC9D00AB5400A100000000DE00AE538D
:100B700000DC9D00AB5400A100000000DA00A85981
:100B800000D8A200AB5400A600000000D600A25F6F
:100B900000D4A700AB5400AB00000000D2009C655D
:100BA00000D0AC00AB5400B000000000CE00966B4B
:100BB00000CCB100AB5400B500000000CA00907139
:100BC00000C8B500AB5400B900000000CA00907125
:100BD00000C8B500AB5400B900000000CE00966B11
:100BE00000CCB100AB5400B500000000D2009C6501
:100BF00000D0AC00AB5400B000000000D600A25FF3
:100C000000D4A700AB5400AB00000000DA00A859E4
:100C100000D8A200AB5400A600000000DE00AE53D6
:100C200000DC9D00AB5400A100000000DE00AE53CC
:100C300000DC9D00AB5400A100000000DA00A859C0
:100C400000D8A200AB5400A600000000D600A25FAE
:100C500000D4A700AB5400AB00000000D2009C659C
:100C600000D0AC00AB5400B000000000CE00966B8A
:100C700000CCB100AB5400B500000000CA00907178
:100C800000C8B500AB5400B900000000CA00907164
:100C900000C8B500AB5400B980000000CD009C65D1
:100CA00000CBB1009F6000B580000000D000A859C3
:100CB00000CEAC00936C00B080000000D300B44DB7
:100CC00000D1A700877800AB80000000D600C041AB
:100CD00000D4A2007B8400A680000000D900CC359F
:100CE00000D79D006F9000A180000000D9BDCC35D9
:100CF000C2D79D006F9000A100000000D6BDC63B8A
:100D0000C2D4A3006B9400A700000000D3BEC04172
:100D1000C3D1A900679800AD00000000D1BFBA4759
:100D2000C4CFAF00639C00B300000000CEC0B44D40
:100D3000C5CCB5005FA000B900000000CBC1AE5328
:100D4000C6C9BB005BA400BF00000000C500AD54D5
:100D500000C3C40052AD00C8A5000000CC00AD51D6
:100D600000C3C40055B400CFA5000000D200AD4EB2
:100D700000C2C30058BA00D5A5000000D100A94C9C
:100D800000C1C2005BBD00D4A5000000C900A34A99
:100D900000C0C1005EBB00CCA5000000C0009D48A3
:100DA00000BEBF0062B900C3A5000000C0009D489E
:100DB00000BEBF0062B900C3A5000000C200A04889
:100DC00000C3C4005DB700C5A5000000C300A34870
:100DD00000C8C90059B500C6A5000000C400A64857
:100DE00000CCCD0055B300C7A5000000C400A94940
:100DF00000D0D10050B100C7A5000000C500AC4B29
:100E000000D3D4004CAF00C8A5000000C500AF4E11
:100E100000D3D40049AC00C8A5000000C400B15202
:100E200000D0D10047A900C7A5000000C400B357F7
:100E300000CCCD0046A600C7A5000000C300B55BEE
:100E400000C8C90046A300C6A5000000C200B75FE5
:100E500000C3C40046A000C5A5000000C000B964DE
:100E600000BEBF00469D00C3A5000000C000B964DD
:100E700000BEBF00469D00C3A5000000C500B961CB
:100E800000C0C10048A200C8A5000000CA00B95EA9
:100E900000C1C2004AA600CDA5000000CE00B95B8B
:100EA00000C2C3004CAA00D1A5000000D200B8586F
:100EB00000C2C3004EAF00D5A5000000D500B65556
:100EC00000C3C40050B300D8A5000000D500B35241
:100ED00000C3C40053B600D8A5000000D200AF5034
:100EE00000C2C30056B800D5A5000000CE00AA4E2F
:100EF00000C2C30059B900D1A5000000CA00A64C29
:100F000000C1C2005CB900CDA5000000C500A24A26
:100F100000C0C1005FB900C8A5000000A3009D6427
:100F200000A100000000000000000000AF00A35E70
:100F300000AD00000000000000000000B800A75A4B
:100F400000B600000000000000000000C100AB5629
:100F500000BF00000000000000000000C800AF5209
:100F600000C600000000000000000000CF00B24FEB
:100F700000CD00000000000000000000CF00B24FD4
:100F800000CDA2C06EA2C0A67A800000C800AF52F9
:100F900000C6A2B965AAB9A670800000C100AB5610
:100FA00000BFA2B65EAEB6A66B800000B800A75A1E
:100FB00000B6A2B258B2B2A666800000AF00A35E2F
:100FC00000ADA2AF51B6AFA661800000A3009D6442
:100FD00000A1A2AB47BCABA65C80000080B344BDBF
:100FE000B87E0000000000008000000000CF00007C
:100FF000D4000000000000007D00000000B40000EC
:10100000B9000000000000007900000000CF0000DF
:10101000D4000000000000007600000000B40000D2
:10102000B9000000000000007200000000CF0000C6
:10103000D4000000000000006E00000000B40000BA
:10104000B9000000000000006B00000000CF0000AD
:10105000D4000000000000006700000000B40000A1
:10106000B9000000000000006300000000CF000095
:10107000D4000000000000006000000000B4000088
:10108000B9000000000000005C00000000B3000098
:10109000B8000000000000008000000000CF000049
:1010A000D4000000000000007D00000000B400003B
:1010B000B9000000000000007900000000CF00002F
:1010C000D4000000000000007600000000B4000022
:1010D000B9000000000000007200000000CF000016
:1010E000D4000000000000006E00000000B400000A
:1010F000B9000000000000006B00000000CF0000FD
:10110000D4000000000000006700000000B40000F0
:10111000B9000000000000006300000000CF0000E4
:10112000D4000000000000006000000000B40000D7
:10113000B9000000000000005C00000080C144BD58
:10114000C87E0000000000008000000000C0000019
:10115000CA000000000000007D00000000BF000089
:10116000CB000000000000007900000000BE00007D
:10117000CD000000000000007600000000BD00006F
:10118000CF000000000000007200000000BD000061
:10119000D0000000000000006E00000000BD000054
:1011A000CB000000000000006B00000000BE00004B
:1011B000CA000000000000006700000000BF00003F
:1011C000C9000000000000006300000000C0000033
:1011D000C8000000000000006000000000C1000026
:1011E000C7000000000000005C00000080C144BD9A
:1011F000C67E0000000000008000000000C2000069
:10120000C6000000000000007D00000000C30000D8
:10121000C5000000000000007900000000C40000CC
:10122000C4000000000000007600000000C50000BF
:10123000C3000000000000007200000000C60000B3
:10124000C2000000000000006E00000000C60000A8
:10125000C2000000000000006B00000000C600009B
:10126000C2000000000000006700000000C5000090
:10127000C3000000000000006300000000C4000084
:10128000C4000000000000006000000000C3000077
:10129000C5000000000000005C00000000C200006B
:1012A000C6000000000000000000000000C10000B7
:1012B000C6000000000000000000000000C10000A7
:1012C000C8000000000000000000000000C0000096
:1012D000CA000000000000000000000000BF000085
:1012E000CB000000000000000000000000BE000075
:1012F000CD000000000000000000000000BD000064
:10130000CF000000000000000000000000BD000051
:10131000D0000000000000000000000000BD000040
:10132000CB000000000000000000000000BE000034
:10133000CA000000000000000000000000BF000024
:10134000C9000000000000000000000000C0000014
:10135000C8000000000000000000000000C1000004
:10136000C7000000000000000000000000C10000F5
:10137000C6000000000000000000000000C20000E5
:10138000C6000000000000000000000000C30000D4
:10139000C5000000000000000000000000C40000C4
:1013A000C4000000000000000000000000C50000B4
:1013B000C3000000000000000000000000C60000A4
:1013C000C2000000000000000000000000C6000095
:1013D000C2000000000000000000000000C6000085
:1013E000C2000000000000000000000000C5000076
:1013F000C3000000000000000000000000C4000066
:10140000C4000000000000000000000000C3000055
:10141000C5000000000000000000000000C2000045
:10142000C6000000000000000000000000C1000035
:10143000C6000000000000000000000000C1000025
:10144000C8000000000000000000000000C0000014
:10145000CA000000000000000000000000BF000003
:10146000CB000000000000000000000000BE0000F3
:10147000CD000000000000000000000000BD0000E2
:10148000CF000000000000000000000000BD0000D0
:10149000D0000000000000000000000000BD0000BF
:1014A000CB000000000000000000000000BE0000B3
:1014B000CA000000000000000000000000BF0000A3
:1014C000C9000000000000000000000000C0000093
:1014D000C8000000000000000000000000C1000083
:1014E000C7000000000000000000000000C1000074
:1014F000C6000000000000000000000088AE51B0EF
:10150000B3860000000000000000000090A35CA56E
:10151000A88E000000000000000000009899689963
:101520009E9600000000000000000000A08E748D58
:10153000939E00000000000000000000A78480814E
:1015400089A500000000000000000000B0798C7543
:101550007EAE0000000000000000000000790000E6
:101560007E00000000000000000000000084000079
:10157000890000000000000000000000008E000054
:10158000930000000000000000000000009900002F
:101590009E000000000000000000000000A300000A
:1015A000A8000000000000000000000000AE0000E5
:1015B000B3000000000000000000000000AE0000CA
:1015C000B3000000000000000000000000A30000C5
:1015D000A8000000000000000000000000990000CA
:1015E0009E0000000000000000000000008E0000CF
:1015F00093000000000000000000000000840000D4
:1016000089000000000000000000000000790000D8
:101610007E000000000000000000000000790000D3
:101620007E000000000000000000000000840000B8
:10163000890000000000000000000000008E000093
:10164000930000000000000000000000009900006E
:101650009E000000000000000000000000A3000049
:10166000A8000000000000000000000000AE000024
:10167000B3000000000000000000000000AE000009
:10168000B3000000000000000000000000A3000004
:10169000A800000000000000000000000099000009
:1016A0009E0000000000000000000000008E00000E
:1016B0009300000000000000000000000084000013
:1016C0008900000000000000000000000079000018
:1016D0007E00000000000000000000000079000013
:1016E0007E000000000000000000000000840000F8
:1016F000890000000000000000000000008E0000D3
:1017000093000000000000000000000000990000AD
:101710009E000000000000000000000000A3000088
:10172000A8000000000000000000000000AE000063
:10173000B3000000000000000000000099008C755C
:101740000097000000000000000000009D00907164
:10175000009B00000000000000000000A000946D4D
:10176000009E00000000000000000000A200986938
:1017700000A000000000000000000000A3009B6625
:1017800000A100000000000000000000A3009D6414
:1017900000A10000000000000000000000000000A8
:1017A0000000AAAB45BEABAE6B800000000000009D
:1017B0000000B2AF40C2AFB6688000000000000079
:1017C0000000BBB23AC7B2BF658000000000000055
:1017D0000000C3B635CBB6C7628000000000000031
:1017E0000000CBB930D0B9CF5F800000000000000E
:1017F0000000D3C32AD5C3D75C800000A300936E3A
:1018000000A100000000000000000000A300887993
:1018100000A100000000000000000000A3007D8483
:1018200000A100000000000000000000A300728F73
:1018300000A100000000000000000000A300679A63
:1018400000A100000000000000000000A3005CA553
:1018500000A100000000000000000000A3009D6443
:1018600000A1A200629D00A600000000AF00A35EE0
:1018700000ADAE005CA300B200000000B800A75AA3
:1018800000B6B70058A700BB00000000C100AB566F
:1018900000BFC00054AB00C400000000C800AF523D
:1018A00000C6C70050AF00CB00000000CF00B24F11
:1018B00000CDCE004DB200D200000000CF00B24FEC
:1018C00000CDCE004DB200D200000000C800AF52E3
:1018D00000C6C70050AF00CB00000000C100AB56EF
:1018E00000BFC00054AB00C400000000B800A75AFD
:1018F00000B6B70058A700BB00000000AF00A35E11
:1019000000ADAE005CA300B200000000A3009D6427
:1019100000A1A200629D00A600000000A3009D643B
:1019200000A1A200629D00A600000000A3009B662B
:1019300000A1A2005FA000A600000000A20098691C
:1019400000A0A1005DA200A500000000A000956C11
:10195000009E9F005CA300A3000000009E00917009
:10196000009C9D005AA500A1000000009A008D7403
:10197000009899005AA5009D000000009A008D74FF
:10198000009899005AA5009D000000009A008D70F3
:1019900000A099005AA5009D000000009A008D6DDE
:1019A00000A899005AA5009D000000009A008D6AC9
:1019B00000B099005AA5009D000000009A008D66B5
:1019C00000B899005AA5009D000000009A008D63A0
:1019D00000C099005AA5009D000000009A008D6388
:1019E00000C099005AA5009D000000009A008D904B
:1019F00000A899005AA5009D000000009A008D9053
:101A000000A899005AA5009D000000009A008D9042
:101A100000A899005AA5009D000000009A008D9032
:101A200000A899005AA5009D000000009A008D9022
:101A300000A899005AA5009D000000009A008D9012
:101A400000A899005AA5009D000000009A008D8C06
:101A500000A599005AA5009D000000009A008D89FC
:101A600000A299005AA5009D000000009A008D85F3
:101A7000009F99005AA5009D000000009A008D82E9
:101A8000009C99005AA5009D000000009A008D7FDF
:101A9000009999005AA5009D000000009A008D74DD
:101AA000009899005AA5009D000000009E009170CA
:101AB000009C9D005AA500A100000000A000956CAC
:101AC000009E9F005CA300A300000000A200986994
:101AD00000A0A1005DA200A500000000A3009B667D
:101AE00000A1A2005FA000A600000000A3009D646A
:101AF00000A1A200629D00A600000000A3009D645A
:101B000000A1A200629D00A600000000A3009B6649
:101B100000A1A2005FA000A600000000A20098693A
:101B200000A0A1005DA200A500000000A000956C2F
:101B3000009E9F005CA300A3000000009E00917027
:101B4000009C9D005AA500A1000000009A008D7421
:101B5000009899005AA5009D000000009A008D741D
:101B6000009899005AA5009D00000000A200917401
:101B7000009899005AA5009D00000000AA009474E6
:101B8000009899005AA5009D00000000B2009774CB
:101B9000009899005AA5009D00000000BA009B74AF
:101BA000009899005AA5009D00000000C2009E7494
:101BB000009899005AA5009D00000000C2009E7484
:101BC000009899005AA5009D00000000AA007174B9
:101BD000009899005AA5009D00000000AA007174A9
:101BE000009899005AA5009D00000000AA00717499
:101BF000009899005AA5009D00000000AA00717489
:101C0000009899005AA5009D00000000AA00717478
:101C1000009899005AA5009D00000000AA00717468
:101C2000009899005AA5009D00000000A700757457
:101C3000009899005AA5009D00000000A400787447
:101C4000009899005AA5009D00000000A1007C7436
:101C5000009899005AA5009D000000009E007F7426
:101C6000009899005AA5009D000000009B00827416
:101C7000009899005AA5009D000000009A008D74FC
:101C8000009899005AA5009D000000009E009170E8
:101C9000009C9D005AA500A100000000A000956CCA
:101CA000009E9F005CA300A300000000A2009869B2
:101CB00000A0A1005DA200A500000000A3009B669B
:101CC00000A1A2005FA000A600000000A3009D6488
:101CD00000A1A200629D00A600000000A3009D6478
:101CE00000A100000000000000000000B200A55CA0
:101CF00000B000000000000000000000BE00AA5775
:101D000000BC00000000000000000000C800AF524E
:101D100000C600000000000000000000D100B34E2B
:101D200000CF00000000000000000000DA00B74A09
:101D300000D80000000000000000000000000000CB
:101D400000000000009DC3A600000000000000008D
:101D50000000000000AFC2D400000000000000003E
:101D60000000000000B1C1F200000000000000000F
:101D70000000000000AAC0F0000000000000000009
:101D80000000000000A2BFD0000000000000000022
:101D900000000000008CBF9C00000000000000005C
:101DA0000000A2C36200000000000000000000006C
:101DB0000000D0C250000000000000000000000041
:101DC0000000EEC14E000000000000000000000016
:101DD0000000ECC055000000000000000000000002
:101DE0000000CCBF5D00000000000000000000000B
:101DF000000098BF7300000000000000DA00B74A3E
:101E000000D800000000000000000000D100B34E28
:101E100000CF00000000000000000000C800AF522A
:101E200000C600000000000000000000BE00AA572D
:101E300000BC00000000000000000000B200A55C33
:101E400000B000000000000000000000A3009D643E
:101E500000A100000000000000000000A3009D643D
:101E600000A100000000000000000000B200A55C1E
:101E700000B000000000000000000000BE00AA57F3
:101E800000BC00000000000000000000C800AF52CD
:101E900000C600000000000000000000D100B34EAA
:101EA00000CF00000000000000000000DA00B74A88
:101EB00000D800000000000000000000DA00B74A6F
:101EC00000D800000000000000000000D100B34E68
:101ED00000CF00000000000000000000C800AF526A
:101EE00000C600000000000000000000BE00AA576D
:101EF00000BC00000000000000000000B200A55C73
:101F000000B000000000000000000000A3009D647D
:101F100000A100000000000000000000A3009D647C
:101F200000A100000000000000000000B200A55C5D
:101F300000B000000000000000000000BE00AA5732
:101F400000BC00000000000000000000C800AF520C
:101F500000C600000000000000000000D100B34EE9
:101F600000CF00000000000000000000DA00B74AC7
:101F700000D800000000000000000000DA00B74AAE
:101F800000D800000000000000000000D100B34EA7
:101F900000CF00000000000000000000C800AF52A9
:101FA00000C600000000000000000000BE00AA57AC
:101FB00000BC00000000000000000000B200A55CB2
:101FC00000B000000000000000000000A3009D64BD
:101FD00000A100000000000000000000A3009D64BC
:101FE00000A100000000000000000000B200A55C9D
:101FF00000B000000000000000000000BE00AA5772
:1020000000BC00000000000000000000C800AF524B
:1020100000C600000000000000000000D100B34E28
:1020200000CF00000000000000000000DA00B74A06
:1020300000D800000000000000000000DA00B74AED
:1020400000D800000000000000000000D100B34EE6
:1020500000CF00000000000000000000C800AF52E8
:1020600000C600000000000000000000BE00AA57EB
:1020700000BC00000000000000000000B200A55CF1
:1020800000B000000000000000000000A3009D64FC
:1020900000A100000000000000000000A3009D64FB
:1020A00000A100000000000000000000B200A55CDC
:1020B00000B000000000000000000000BE00AA57B1
:1020C00000BC00000000000000000000C800AF528B
:1020D00000C600000000000000000000D100B34E68
:1020E00000CF00000000000000000000DA00B74A46
:1020F00000D8000000000000000000000000000008
:1021000000000000008CBF9C0000000000000000E8
:102110000000000000A2C0D000000000000000008D
:102120000000000000AAC1F0000000000000000054
:102130000000000000B1C2F200000000000000003A
:102140000000000000AFC3D4000000000000000049
:1021500000000000009DC3A6000000000000000079
:10216000000098BF730000000000000000000000A5
:102170000000CCC05D000000000000000000000076
:102180000000ECC15500000000000000000000004D
:102190000000EEC24E000000000000000000000041
:1021A0000000D0C35000000000000000000000004C
:1021B0000000A2C36200000000000000DA00B74A7D
:1021C00000D800000000000000000000D100B34E65
:1021D00000CF00000000000000000000C800AF5267
:1021E00000C600000000000000000000BE00AA576A
:1021F00000BC00000000000000000000B200A55C70
:1022000000B000000000000000000000A3009D647A
:1022100000A100000000000000000000A3009DCB12
:1022200000AEA200623600B300000000A3009DCB08
:1022300000AEA200623600B300000000B500A6CBDD
:1022400000AEB400593600B300000000B500A6CBC4
:1022500000AEB400593600B300000000C300ADCB9F
:1022600000AEC200523600B300000000C300ADCB88
:1022700000AEC200523600B300000000CF00B2CB67
:1022800000AECE004D3600B300000000CF00B2CB50
:1022900000AECE004D3600B300000000DA00B7CB30
:1022A00000AED900483600B300000000DA00B7CB1A
:1022B00000AED900483600B300000000E400BBCBFC
:1022C00000AEE300443600B300000000E400BBCBE6
:1022D00000AEE300443600B3000000000000000040
:1022E000BA00000000000000000000000000000034
:1022F000AE00000000000000000000000000000030
:10230000A20000000000000000000000000000002B
:102310009600000000000000000000000000000027
:102320008B00000000000000000000000000000022
:102330007E0000000000000000000000000000001F
:102340008B00000000000000000000000000000002
:1023500096000000000000000000000000000000E7
:10236000A2000000000000000000000000000000CB
:10237000AE000000000000000000000000000000AF
:10238000BA00000000000000000000000000000093
:10239000C600000000000000000000000000005027
:1023A00000AE000000B100B30000000000000050CB
:1023B00000AE000000B100B30000000000000050BB
:1023C00000AE000000B100B30000000000000050AB
:1023D00000AE000000B100B300000000000000509B
:1023E00000AE000000B100B300000000000000508B
:1023F00000AE000000B100B300000000000000507B
:1024000000AE000000B100B300000000000000506A
:1024100000AE000000B100B300000000000000505A
:1024200000AE000000B100B300000000000000504A
:1024300000AE000000B100B300000000000000503A
:1024400000AE000000B100B300000000000000502A
:1024500000AE000000B100B3000000000000006406
:1024600000A10000009D00A6000000000000005B2D
:1024700000B3000000A600B80000000000000054F7
:1024800000C1000000AD00C6000000000000004FC9
:1024900000CD000000B200D2000000000000004AA1
:1024A00000D8000000B700DD00000000000000467A
:1024B00000E2000000BB00E700000000E400BB46B3
:1024C00000E2E30044BB00E700000000DA00B74A86
:1024D00000D8D90048B700DD00000000CF00B24F9F
:1024E00000CDCE004DB200D200000000C300AD54BC
:1024F00000C1C20052AD00C600000000B500A65BDE
:1025000000B3B40059A600B800000000A3009D6409
:1025100000A1A200629D00A600000000B000366489
:1025200000A1AF00C99D00A600000000B000366405
:1025300000A1AF00C99D00A600000000B000365BFE
:1025400000B3AF00C9A600B800000000B000365BC1
:1025500000B3AF00C9A600B800000000B0003654B8
:1025600000C1AF00C9AD00C600000000B000365485
:1025700000C1AF00C9AD00C600000000B000364F7A
:1025800000CDAF00C9B200D200000000B000364F4D
:1025900000CDAF00C9B200D200000000B000364A42
:1025A00000D8AF00C9B700DD00000000B000364A17
:1025B00000D8AF00C9B700DD00000000B00036460B
:1025C00000E2AF00C9BB00E700000000B0003646E3
:1025D00000E2AF00C9BB00E70000000000B500004A
:1025E00000000000000000000000000000A9000042
:1025F000000000000000000000000000009D00003E
:102600000000000000000000000000000091000039
:102610000000000000000000000000000086000034
:102620000000000000000000000000000079000031
:102630000000000000000000000000000086000014
:1026400000000000000000000000000000910000F9
:10265000000000000000000000000000009D0000DD
:1026600000000000000000000000000000A90000C1
:1026700000000000000000000000000000B50000A5
:1026800000000000000000000000000000C1000089
:10269000000000000000000000000000B000B100D9
:1026A0000000AF004E00000000000000B000B100CC
:1026B0000000AF004E00000000000000B000B100BC
:1026C0000000AF004E00000000000000B000B100AC
:1026D0000000AF004E00000000000000B000B1009C
:1026E0000000AF004E00000000000000B000B1008C
:1026F0000000AF004E00000000000000B000B1007C
:102700000000AF004E00000000000000B000B1006B
:102710000000AF004E00000000000000B000B1005B
:102720000000AF004E00000000000000B000B1004B
:102730000000AF004E00000000000000B000B1003B
:102740000000AF004E00000000000000B000B1002B
:102750000000AF004E00000000000000A3009D003C
:102760000000A2006200000000000000B500A6000A
:102770000000B4005900000000000000C300AD00DC
:102780000000C2005200000000000000CF00B200B4
:102790000000CE004D00000000000000DA00B7008D
:1027A0000000D9004800000000000000E400BB0069
:1027B0000000E3004400000000000000E400BB460D
:1027C00000E2E30044BB00E700000000DA00B74A83
:1027D00000D8D90048B700DD00000000CF00B24F9C
:1027E00000CDCE004DB200D200000000C300AD54B9
:1027F00000C1C20052AD00C600000000B500A65BDB
:1028000000B3B40059A600B800000000A3009D6406
:1028100000A1A200629D00A600000000A3009D642C
:1028200000A1A200629D00A600000000AF00A35E10
:1028300000ADB1005AA500B500000000B900A859CC
:1028400000B7BD0055AA00C100000000BE00AA5795
:1028500000BCC70050AF00CB00000000B500A65B75
:1028600000B3D0004CB300D400000000AA00A16067
:1028700000A8D90048B700DD00000000A3009D6457
:1028800000A1D90048B700DD00000000AF00A35E42
:1028900000ADD0004CB300D400000000B900A8592E
:1028A00000B7C70050AF00CB00000000BE00AA5721
:1028B00000BCBD0055AA00C100000000B500A65B29
:1028C00000B3B1005AA500B500000000AA00A16045
:1028D00000A8A200629D00A6000000009F005C000E
:1028E000000000000000000000000000A7005C00E5
:1028F000000000000000000000000000B0005C00CC
:10290000000000000000000000000000B7005C00B4
:10291000000000000000000000000000BF005C009C
:10292000000000000000000000000000C8005C0083
:102930000000000000000000000000009F005C009C
:10294000000000000000000000000000A7005C0084
:10295000000000000000000000000000B0005C006B
:10296000000000000000000000000000B7005C0054
:10297000000000000000000000000000BF005C003C
:10298000000000000000000000000000C8005C0023
:102990000000000000000000000000009F005C003C
:1029A000000000000000000000000000A7005C0024
:1029B000000000000000000000000000B0005C000B
:1029C000000000000000000000000000B7005C00F4
:1029D000000000000000000000000000BF005C00DC
:1029E000000000000000000000000000C8005C00C3
:1029F0000000000000000000000000009F005C00DC
:102A0000000000000000000000000000A7005C00C3
:102A1000000000000000000000000000B0005C00AA
:102A2000000000000000000000000000B7005C0093
:102A3000000000000000000000000000BF005C007B
:102A4000000000000000000000000000C8005C0062
:102A5000000000000000000000000000A3009D0036
:102A6000000000000000000000000000A3009D64C2
:102A700000A1A200629D00A600000000A300A061CA
:102A800000A1A20064AA00BB00000000A200A25F97
:102A900000A0A10067B500CA00000000A000A45D6E
:102AA000009E9F006BB800C9000000009D00A55C5F
:102AB000009B9C006FB100B7000000009900A55C6E
:102AC0000097980073A5009C000000009900A55C89
:102AD0000097980073000000000000009D00A55CB6
:102AE000009B9C006F00000000000000A000A45D9F
:102AF000009E9F006B00000000000000A200A25F8B
:102B000000A0A1006700000000000000A300A06179
:102B100000A1A2006400000000000000A3009D646A
:102B200000A1A2006200000000000000000000649C
:102B300000A1000000000000000000000000005D97
:102B400000B6000000000000000000000000005A75
:102B500000C5000000000000000000000000005E52
:102B600000C400000000000000000000000000673A
:102B700000B200000000000000000000000000752E
:102B8000009700000000000000000000A3009D75F9
:102B90000097A20062A5009C00000000A300A071A5
:102BA000009BA20064A500A000000000A200A26D8E
:102BB000009EA10067A400A300000000A000A4697B
:102BC00000A09F006BA200A5000000009D00A5666C
:102BD00000A19C006FA000A6000000009900A56461
:102BE00000A19800739D00A60000000000000000F6
:102BF00000009800730000000000000000000000CA
:102C00000000A8006A0000000000000000000000B2
:102C10000000B3006300000000000000000000009E
:102C20000000BC005C00000000000000000000008C
:102C30000000C4005600000000000000000000007A
:102C40000000CB0050000000000000000000000069
:102C50000000CB004D00000000000000000000005C
:102C60000000C4004D000000000000000000000053
:102C70000000BC004E00000000000000000000004A
:102C80000000B30050000000000000000000000041
:102C90000000A80054000000000000000000000038
:102CA000000098005A000000000000009900A500F4
:102CB000000000000000000000000000A900AB00C0
:102CC000000000000000000000000000B400AF00A1
:102CD000000000000000000000000000BD00B10086
:102CE000000000000000000000000000C500B2006D
:102CF000000000000000000000000000CC00B20056
:102D0000000000000000000000000000CC00AF0048
:102D1000000000000000000000000000C500A90045
:102D2000000000000000000000000000BD00A30043
:102D3000000000000000000000000000B4009C0043
:102D4000000000000000000000000000A900950045
:102D500000000000000000000000000099008C004E
:102D600000000000000000000000000099008C64DA
:102D700000A198005A9D00A6000000009D009061EF
:102D800000A19C005A9B00A600000000A000945FD8
:102D900000A09F005B9800A500000000A200985DC5
:102DA000009EA1005D9400A300000000A3009B5CB6
:102DB000009BA2005F9000A000000000A3009D5CAB
:102DC0000097A200628C009C000000000000000040
:102DD00000000000009D00A60000000000000000B0
:102DE0000000000000AA00BB00000000000000007E
:102DF0000000000000B500CA000000000000000054
:102E00000000000000B800C9000000000000000041
:102E10000000000000B100B700000000000000004A
:102E20000000000000A5009C000000000000000061
:102E30000000000000A5009C000000000000000051
:102E40000000000000A500A000000000000000003D
:102E50000000000000A400A300000000000000002B
:102E60000000000000A200A500000000000000001B
:102E70000000000000A000A600000000000000000C
:102E800000000000009D00A600000000000000649B
:102E900000A1000000000000000000000000005D34
:102EA00000B6000000000000000000000000005A12
:102EB00000C5000000000000000000000000005EEF
:102EC00000C40000000000000000000000000067D7
:102ED00000B20000000000000000000000000075CB
:102EE00000970000000000000000000000000075D6
:102EF00000970000000000000000000000000071CA
:102F0000009B000000000000000000000000006DB9
:102F1000009E0000000000000000000000000069AA
:102F200000A000000000000000000000000000669B
:102F300000A100000000000000000000000000648C
:102F400000A100000000000000000000A3C19D647B
:102F5000C6A1A2C3629DC3A600640000A3C09E5C7C
:102F6000C5B0B1C25A9EC2A600000000A3BF9F55C3
:102F7000C4BCBDC1539FC1A600000000A3BEA054A5
:102F8000C3BCBDC052A0C0A600000000A3BDA05994
:102F9000C2B0B1BF57A0BFA600000000A2BDA16093
:102FA000C2A0A1BF5EA1BFA500000000A2BDA1609C
:102FB000C2A0A1BF5EA1BFA500000000B2BEA86173
:102FC000C3A1A2C05FA8C0B500000000BEBFAD6134
:102FD000C4A1A2C15FADC1C100000000BEC0AC620F
:102FE000C5A1A2C260ACC2C100000000B2C1A5630D
:102FF000C6A1A2C361A5C3B500000000A3C19D6422
:10300000C6A1A2C3629DC3A600800000A3BF9D64A9
:10301000C4A1A2C1629DC1A600640000A3BD9F5BC4
:10302000C2B0B1BF599FBFA600000000A3BBA05310
:10303000C0BCBDBD51A0BDA600000000A2B9A252F7
:10304000BEBBBCBB50A2BBA500000000A1B8A356EC
:10305000BDAEAFBA54A3BAA400000000A0B5A45DF1
:10306000BA9E9FB75BA4B7A300000000A0B8A45D00
:10307000BD9E9FBA5BA4BAA300000000B0B9AB5ECE
:10308000BE9FA0BB5CABBBB300000000BDBBAF5F8D
:10309000C0A0A1BD5DAFBDC000000000BEBDAE615F
:1030A000C2A1A2BF5FAEBFC100000000B2BFA66256
:1030B000C4A1A2C160A6C1B500000000A3C19D6467
:1030C000C6A1A2C3629DC3A600800000A3C19D64E7
:1030D000C6A1A2C3629DC3A6009C0000B2C0A563A6
:1030E000C5A1A2C261A5C2B500000000BEBFAC620E
:1030F000C4A1A2C160ACC1C100000000BEBEAD61F0
:10310000C3A1A2C05FADC0C100000000B2BDA861F4
:10311000C2A1A2BF5FA8BFB500000000A2BDA16010
:10312000C2A0A1BF5EA1BFA500000000A2BDA1601A
:10313000C2A0A1BF5EA1BFA500000000A3BEA05910
:10314000C3B0B1C057A0C0A600000000A3BFA054E8
:10315000C4BCBDC152A0C1A600000000A3C09F55C1
:10316000C5BCBDC2539FC2A600000000A3C19E5CA7
:10317000C6B0B1C35A9EC3A600000000A3C19D649F
:10318000C6A1A2C3629DC3A600800000A3BF9D6428
:10319000C4A1A2C1629DC1A6009C0000B2BDA662EE
:1031A000C2A1A2BF60A6BFB500000000BEBBAD615A
:1031B000C0A1A2BD5FADBDC100000000BDB9AF6040
:1031C000BEA0A1BB5EAFBBC000000000B1B8AA5F4B
:1031D000BDA0A1BA5DAABAB400000000A1B5A35E6B
:1031E000BA9FA0B75CA3B7A400000000A1B8A35E7B
:1031F000BD9FA0BA5CA3BAA400000000A2B9A25768
:10320000BEAFB0BB55A2BBA500000000A2BBA1523F
:10321000C0BBBCBD50A1BDA500000000A3BDA05413
:10322000C2BCBDBF52A0BFA600000000A3BF9F5BF1
:10323000C4B0B1C1599FC1A600000000A3C19D64E4
:10324000C6A1A2C3629DC3A600800000A3C19D6465
:10325000C6A1A2C4629DC3A680800000A3C19D64D4
:10326000C6A1A2C4629DC3A680800000A3C19D64C4
:10327000C6A1A2C4629DC3A680800000A3C19D64B4
:10328000C6A1A2C4629DC3A680800000A3C19D64A4
:10329000C6A1A2C4629DC3A680800000C500AD5433
:1032A00000C3C40052AD00C8A5000000CC00AD5062
:1032B00000C2C30055B400CFA5000000D200AB4D42
:1032C00000C2C30059BB00D5A5000000D100A74B28
:1032D00000C0C1005DBF00D4A5000000C800A04828
:1032E00000BEBF0061BD00CBA5000000BE009A4734
:1032F00000BCBD0065BA00C1A5000000BE009A4731
:1033000000BCBD0065BA00C1A5000000C0009E461B
:1033100000C2C30060B900C3A5000000C200A146FE
:1033200000C7C8005BB700C5A5000000C300A547E3
:1033300000CBCC0056B400C6A5000000C400A849CC
:1033400000CFD00051B200C7A5000000C500AC4BB3
:1033500000D3D4004CAF00C8A5000000C500AF4E9C
:1033600000D3D40049AC00C8A5000000C400B2538B
:1033700000CFD00047A800C7A5000000C300B45884
:1033800000CBCC0045A500C6A5000000C200B75D7B
:1033900000C7C80044A100C5A5000000C000B96274
:1033A00000C2C300449E00C3A5000000BE00BA676F
:1033B00000BCBD00459A00C1A5000000BE00BA6770
:1033C00000BCBD00459A00C1A5000000C400BB635D
:1033D00000BEBF00469F00C7A5000000C900BB603B
:1033E00000C0C10048A400CCA5000000CD00BA5C1C
:1033F00000C1C2004BA900D0A5000000D100B859FF
:1034000000C2C3004DAE00D4A5000000D500B655E3
:1034100000C3C40050B300D8A5000000D500B352CB
:1034200000C3C40053B600D8A5000000D100AE4FC1
:1034300000C2C30057B800D4A5000000CD00A94DBC
:1034400000C1C2005ABA00D0A5000000C900A44AB9
:1034500000C0C1005EBB00CCA5000000C4009F48B6
:1034600000BEBF0061BB00C7A5000000BE009A47B8
:1034700000BCBD0065BA00C1A5000000BE009A47AF
:1034800000BCBD0065BA00C1A5000000C0009E449C
:1034900000C6C7005FB900C3A5000000C200A24279
:1034A00000CFD00058B600C5A5000000C400A64655
:1034B00000D0D10054B400C7A5000000C400AA4D3C
:1034C00000CACB0052B100C7A5000000C500AD5432
:1034D00000C3C40052AD00C8A5000000A3009D6455
:1034E00000A1A200629D00A600000000A3009D6450
:1034F00000A1AE005CA300B200000000A3009D6428
:1035000000A1B70058A700BB00000000A3009D6405
:1035100000A1C00054AB00C400000000A3009D64E3
:1035200000A1C70050AF00CB00000000A3009D64C5
:1035300000A1CE004DB200D200000000A3009D64A7
:1035400000A1CE004DB200D200000000A600976896
:1035500000A4C60045BA00CA00000000A800916D92
:1035600000A6BE003DC200C200000000AA008B728F
:1035700000A8B60035CA00BA00000000AD0085778B
:1035800000ABAE002DD200B200000000AF007F7C87
:1035900000ADA60025DA00AA00000000AF007F7C85
:1035A00000ADA60025DA00AA80000000A7007982FD
:1035B00000A5A60025DA00AA8A0000009F007388F3
:1035C000009DA60025DA00AA9300000097006D8EEA
:1035D0000095A60025DA00AA9C0000008F006794E1
:1035E000008DA60025DA00AAA50000008700619AD8
:1035F0000085A60025DA00AAAE0000000000000049
:103600000000A60025DA00AAAE00000000000000BD
:103610000000B00021DE00B4A500000000000000A2
:103620000000BB001DE200BF9C0000000000000085
:103630000000C50019E600C993000000000000006A
:103640000000D00015EA00D48A000000000000004D
:103650000000DA0011EE00DE800000000000000033
:103660000000DA0011EE00DE0000000000000000A3
:103670000000DA001EE100DE000000000000000093
:103680000000DA002CD300DE000000000000000083
:103690000000DA0039C600DE000000000000000073
:1036A0000000DA0046B900DE000000000000000063
:1036B0000000DA0054AB00DE0000000080008C75D2
:1036C000007EDA0054AB00DE000000008C00937036
:1036D000008AD40054AB00D8000000009800996B19
:1036E0000096CE0054AB00D200000000A4009F66FC
:1036F00000A2C80054AB00CC00000000B000A561DF
:1037000000AEC20054AB00C600000000BB00AA5CC3
:1037100000B9BC0054AB00C000000000A3C29D0073
:10372000C80000C3009DC3A600000000A8C3A000FD
:10373000CA0000C200A0C2AB00000000ADC4A200DD
:10374000CB0000C100A2C1B000000000ADC5A200C6
:10375000CD0000C000A2C0B000000000A8C6A000BC
:10376000CF0000BF00A0BFAB00000000A3C69D00BB
:10377000D00000BF009DBFA60000000000C600648E
:10378000CBA1A2BF6200BF000000000000C5006224
:10379000CAA3A4C06000C0000000000000C4006113
:1037A000C9A5A6C15F00C1000000000000C3006100
:1037B000C8A7A8C25F00C2000000000000C20060ED
:1037C000C7A9AAC35E00C3000000000000C1005FDB
:1037D000C6ABACC35D00C3000000000000C1005FC9
:1037E000C6ABACC45D00C5000000000000C00060B6
:1037F000C5A9AAC55E00C7000000000000BF0061A7
:10380000C4A7A8C65F00C8000000000000BE006199
:10381000C3A5A6C75F00CA000000000000BD00628B
:10382000C2A3A4C86000CC000000000000BD00647A
:10383000C2A1A2C86200CD0000000000A3BD9D008F
:10384000C20000C8009DC8A600000000A5BE9F00E1
:10385000C30000C7009FC7A800000000A7BFA000CA
:10386000C40000C600A0C6AA00000000A9C0A000B5
:10387000C50000C500A0C5AC00000000ABC1A100A0
:10388000C60000C400A1C4AE00000000ADC1A2008B
:10389000C60000C300A2C3B000000000ADC2A20079
:1038A000C80000C300A2C3B000000000ABC3A10069
:1038B000CA0000C200A1C2AE00000000A9C4A0005E
:1038C000CB0000C100A0C1AC00000000A7C5A00053
:1038D000CD0000C000A0C0AA00000000A5C69F0047
:1038E000CF0000BF009FBFA800000000A3C69D003E
:1038F000D00000BF009DBFA60000000000C600640D
:10390000CBA1A2BF6200BF000000000000C50061A3
:10391000CAA6A7C05F00C0000000000000C4005F8E
:10392000C9ABACC15D00C1000000000000C3005F76
:10393000C8ABACC25D00C2000000000000C2006164
:10394000C7A6A7C35F00C3000000000000C1006459
:10395000C6A1A2C36200C30000000000A3C19D0075
:10396000C60000C4009DC5A600000000A8C0A000BD
:10397000C50000C500A0C7AB00000000ADBFA2009D
:10398000C40000C600A2C8B000000000ADBEA20086
:10399000C30000C700A2CAB000000000A8BDA0007C
:1039A000C20000C800A0CCAB00000000A3BD9D0079
:1039B000C20000C8009DCDA60000000000BD00644C
:1039C000C2A1A2C86200C8000000000000BE0062E0
:1039D000C3A3A4C76000C7000000000000BF0061CF
:1039E000C4A5A6C65F00C6000000000000C00061BC
:1039F000C5A7A8C55F00C5000000000000C10060A9
:103A0000C6A9AAC45E00C4000000000000C1005F97
:103A1000C6ABACC35D00C3000000000000C2005F85
:103A2000C8ABACC35D00C3000000000000C3006071
:103A3000CAA9AAC25E00C2000000000000C4006162
:103A4000CBA7A8C15F00C1000000000000C5006155
:103A5000CDA5A6C05F00C0000000000000C6006247
:103A6000CFA3A4BF6000BF000000000000C6006438
:103A7000D0A1A2BF6200BF0000000000A3C69D004D
:103A8000CB0000BF009DBFA600000000A5C59F00A1
:103A9000CA0000C0009FC0A800000000A7C4A0008A
:103AA000C90000C100A0C1AA00000000A9C3A00075
:103AB000C80000C200A0C2AC00000000ABC2A10060
:103AC000C70000C300A1C3AE00000000ADC1A2004A
:103AD000C60000C300A2C3B000000000ADC1A20038
:103AE000C60000C400A2C5B000000000ABC0A10029
:103AF000C50000C500A1C7AE00000000A9BFA0001E
:103B0000C40000C600A0C8AC00000000A7BEA00012
:103B1000C30000C700A0CAAA00000000A5BD9F0006
:103B2000C20000C8009FCCA800000000A3BD9D00FB
:103B3000C20000C8009DCDA60000000000BD0064CA
:103B4000C2A1A2C86200C8000000000000BE00615F
:103B5000C3A6A7C75F00C7000000000000BF005F4A
:103B6000C4ABACC65D00C6000000000000C0005F32
:103B7000C5ABACC55D00C5000000000000C1006120
:103B8000C6A6A7C45F00C4000000000000C1006416
:103B9000C6A1A2C36200C30000000000A3009D6490
:103BA00000A1A200629D00A600000000A3009A6789
:103BB00000A1A2005FA000A600000000A100966B7B
:103BC000009FA0005CA300A4000000009E00917074
:103BD000009C9D005BA400A1000000009E0091706D
:103BE000009C9D005BA400A1000000009E00916A63
:103BF00000A89D005BA400A1000000009E0091654C
:103C000000B49D005BA400A1000000009E00916034
:103C100000C09D005BA400A1000000009E00916018
:103C200000C09D005BA400A1000000009E0091C7A1
:103C3000009C9D005BA400A1000000009E0091C7B5
:103C4000009C9D005BA400A1000000009E0091C7A5
:103C5000009C9D005BA400A1000000009E0091C795
:103C6000009C9D005BA400A1000000009E0091C785
:103C7000009C9D005BA400A1000000009E0091C775
:103C8000009C9D005BA400A1000000009E0091C765
:103C9000009C9D005BA400A1000000009E0091C755
:103CA000009C9D005BA400A1000000009E0091C24A
:103CB00000979D005BA400A1000000009E0091BD44
:103CC00000939D005BA400A1000000009E0091B83D
:103CD000008E9D005BA400A1000000009E0091707A
:103CE000009C9D005BA400A100000000A100966B59
:103CF000009FA0005CA300A400000000A3009A673E
:103D000000A1A2005FA000A600000000A3009D6427
:103D100000A1A200629D00A600000000A3009D6417
:103D200000A1A200629D00A600000000A3009A6707
:103D300000A1A2005FA000A600000000A100966BF9
:103D4000009FA0005CA300A4000000009E009170F2
:103D5000009C9D005BA400A1000000009E009170EB
:103D6000009C9D005BA400A100000000AA009770C9
:103D7000009C9D005BA400A100000000B6009C70A8
:103D8000009C9D005BA400A100000000C200A17087
:103D9000009C9D005BA400A100000000C200A17077
:103DA000009C9D005BA400A1000000009E003A70F2
:103DB000009C9D005BA400A1000000009E003A70E2
:103DC000009C9D005BA400A1000000009E003A70D2
:103DD000009C9D005BA400A1000000009E003A70C2
:103DE000009C9D005BA400A1000000009E003A70B2
:103DF000009C9D005BA400A1000000009E003A70A2
:103E0000009C9D005BA400A1000000009E003A7091
:103E1000009C9D005BA400A1000000009E003A7081
:103E2000009C9D005BA400A10000000099003F7071
:103E3000009C9D005BA400A1000000009500447060
:103E4000009C9D005BA400A1000000009000497050
:103E5000009C9D005BA400A1000000009E009170EA
:103E6000009C9D005BA400A100000000A100966BD7
:103E7000009FA0005CA300A400000000A3009A67BC
:103E800000A1A2005FA000A600000000A3009D64A6
:103E900000A1A200629D00A6000000000000F894AE
:103EA000EE27ECBBF1E0F5BFE5BFE0936C00EBBFA4
:103EB000F8E1F1BDF0E1F1BD8DE0A2E0BB27ED93AB
:103EC0008A95E9F780E090E1A0E0B1E0ED930197F9
:103ED000E9F7ECE9FEE305901590BF01F00130979A
:103EE00051F0A591B5918591959105900D9201970D
:103EF000E1F7FB01F0CFEFEFEDBFE0E1EEBFC0E097
:103F0000D5E00C94831FEE27EBBBEABBE8BBE7BB15
:103F1000E5BBE4BBEEE0E2BBE2E0E1BBEE27E3BFE2
:103F2000E2BFE1BFEFBDE5E0EEBDEE27EDBDECBDCC
:103F3000EBBDEABDE9BDE8BDE0BFE5BDE4BDE3BD65
:103F4000EFE0E0936A00EE27EABFE3E0E9BFE8BFF5
:103F5000E4E0E7BFEE27EBB9E8E1EAB9E6E0E09399
:103F60009500EE27E0939000EFE0E9B9EE27E093AB
:103F70009B00E8E1E0939A00E6E0E0939D00EE27E5
:103F8000E0939800EFE0E0939900E0E8E8B9EE27CD
:103F9000E0BD789478D2FFCF0E942D240E94402368
:103FA000E1E0BE2E0E943B2418950E942D240E9421
:103FB00040232ED30E943B2418950E942D241A934F
:103FC0000A9300E010E00CB10F3F69F410E01530E7
:103FD00040F4A12FBB27A050BB4FEE27EC931F5FEF
:103FE000F6CFCC2459C0AC2DBB27A050BB4F0C93AF
:103FF000C394E5E0EC1519F5E0910405EF93E09129
:104000000105A0910005EA27AF910E945224EF77A5
:10401000E03021F0A0910005A03009F00FC0E1E0F0
:10402000F5E0D080E2E0F5E0E080E0910305E09388
:104030000505CC24E1E0E093060501C0CC242CC0AA
:104040000E942D241A930A9300E010E0681479046A
:1040500018F00E94402320C000E010E00031E0E0B2
:104060001E079CF40E944423E03061F0E02FF12F02
:10407000EA930E944423EA93E0910905F0910A052E
:10408000EA930FD00F5F1F4FE9CFE62DF72D319642
:104090006E2E7F2E5DBC4CBC099119910E943B2471
:1040A00018950A9300E0E981E295E07FEE0FE07E4B
:1040B000AB81EA2B0E2FA23019F4EA81E450EA8397
:1040C000AB81A33019F4EA81E750EA83AB81A430D5
:1040D00011F40E945223AB81A53019F4EA81EC5F00
:1040E000EA83AB81A63019F4EA81E85FEA83AB8109
:1040F000A83019F4EA81E550EA83AB81A93019F4BC
:10410000EA81E250EA83AB81AB3011F40E94522382
:10411000EFEF0E9456230A93A0D285E08A95F1F72B
:10412000EA810E945623EA81E027EF770E94562316
:10413000EE27FF2708813FC0A881B981AF3FEFEF8D
:10414000BE0738F4EFEFFFEFEA1BFB0B4E2E5F2E9E
:1041500002C044245524EE27FF2722960895E881C3
:10416000E03041F40E945D235DBC4CBC66247724A2
:10417000AA2418C0E73069F40E946223EE27FF27C3
:10418000FDBDECBD66247724E1E0AE2EEE27E7BF4F
:1041900009C0E23019F40E94622304C0E33011F434
:1041A0000E945D2361C2EA81FB81E0930705F093E1
:1041B000080588809980249608950E946623ECE47F
:1041C000F2E3FA93EA93E5E0F0E00E947223AA207A
:1041D000F1F357C10E947A230E946623ECEDF4E3C9
:1041E0000E948223AA20F1F34CC1E1E0F0E0E093C9
:1041F0000905F0930A05E0EBF4E0FA93EA930E94D4
:104200009C20ECE5F6E30E948723AA20F1F30E94AC
:104210007A2337C10E946623ECE1F8E20E948C23E6
:10422000AA20F1F30E946623ECEDF8E2FA93EA93F8
:10423000E9E1F0E00E947223AA20F1F30E947A23C0
:1042400020C11A930A9300E010E00E949123ECE948
:10425000F2E30E948C23AA20F1F30E949D230E9486
:10426000572438F4ECEFF2E30E948223AA20F1F302
:10427000F4CFECE7F4E30E948C23AA20F1F3C7C04B
:104280000E946623ECE9FBE30E948223AA20F1F35B
:10429000F8C00E946623ECE1FDE30E948223AA207D
:1042A000F1F3EFC01A930A9300E010E00E9491230B
:1042B000ECE8F0E00E94A423AA20F1F3ECE0F1E0A6
:1042C0000E94A923AA20F1F30E949D23A130E0E0DF
:1042D000BE0738F4ECE0F3E00E94A423AA20F1F337
:1042E00096C0ECE0F2E00E94A923AA20F1F3E6CF09
:1042F0008EC01A930A9300E010E00E949123ECE82C
:10430000F3E00E94A423AA20F1F3ECE0F4E00E9481
:10431000A923AA20F1F30E949D23A130E0E0BE076B
:1043200038F4ECE0F6E00E94A423AA20F1F36FC079
:10433000ECE0F5E00E94A923AA20F1F3E6CF67C0E4
:104340001A930A9300E010E00E949123ECE1F7E356
:104350000E948C23AA20F1F30E949D230E945724DF
:1043600038F4ECE7F7E30E948223AA20F1F3F4CFBC
:10437000ECEFF8E30E948C23AA20F1F348C01A93D3
:104380000A9300E010E00E949123ECE5F9E30E941B
:104390008C23AA20F1F30E949D230E94572438F415
:1043A000ECEBF9E30E948223AA20F1F3F4CFECE3D3
:1043B000FBE30E948C23AA20F1F329C01A930A93ED
:1043C00000E010E00E94AE230E949D230E9457242B
:1043D00048F40E94B523ECE0F0E30E948723AA2072
:1043E000F1F3F2CF14C01A930A9300E010E00E9498
:1043F000AE230E949D230E94572448F40E94B523B7
:10440000ECE8F1E30E948723AA20F1F3F2CF1981AF
:104410000881279608950E946623ECE8F6E00E9442
:10442000BB23AA20F1F32DC00E946623ECE8F9E03B
:10443000FA93EA93ECE3F0E00E947223AA20F1F3EE
:104440000E947A231EC00E946623ECE1F5E20E94DE
:10445000BB23AA20F1F315C00E946623ECE1F2E22F
:104460000E94BB23AA20F1F30CC00E946623ECED4E
:10447000FCE1FA93EA93E4E5F0E00E947223AA20BB
:10448000F1F3239608950E945B2400E010E020E001
:1044900030E0E8EEF3E00E94C0230E94C723E0ED85
:1044A000F7E0FA93EA930E942124BB24BB20F1F3A6
:1044B0000E94CD230E94D8230E945221E4EFF1E014
:1044C0000E94C023E4EFF1E00E94E9230E94F02360
:1044D0000E94F5230E94DE21E4EFF1E00E94C02358
:1044E000E0EBF4E0FA93EA930E9435220E94FE2367
:1044F0000E94D8230E9479210E940124E6E0F0E086
:10450000FA93EA930E94BF210E940124E4E0F0E0C4
:10451000FA93EA930E94A021E4EFF1E00E94C02305
:10452000E4EBF0E00E94E9230E942121E2E0EA931B
:10453000E4EFF1E0FA93EA930E94DD200E940E245A
:104540000E9449210E940E240E944021E4EFF1E0E4
:104550000E94C023E8EEF3E0FA93EA930E942C2233
:104560000E94FE23E4EFF1E00E94C023E8EEF3E0B6
:10457000FA93EA930E9423220E94FE23E4EFF1E0E3
:104580000E94C0230E94F5230E94F023E8E7F5E093
:10459000FA93EA930E9414220E94FE230E9415249B
:1045A000E3E0EA93E8E7F5E0FA93EA930E940B224E
:1045B000E2E0EA93ECEDF5E0FA93EA930E94DD2065
:1045C000E4EFF1E00E94C0230E94F5230E94DE2167
:1045D0000E9415240E9415240E94CD23E2E00E942F
:1045E0001B240E94EA20E8EBFBE0FA93EA930E9486
:1045F0002124EE270E941B240E94F520E3E0EA9389
:10460000E8ECF0E0FA93EA930E94DD2051CF21C05C
:104610000E945B2420E030E02330E0E03E07ACF471
:1046200000E010E00031E0E01E0764F4E02FF12F1D
:10463000EA93EE27EA93E5E0EA930E9451200F5FA8
:104640001F4FF0CF2F5F3F4FE7CF6624772488249A
:1046500099240E94602424960895E0919B00E072C2
:10466000E1F3E881E0939C00219608955F9BFECFE3
:10467000ECB108955D9BFECFE881ECB921960895D9
:10468000E7E0EA930C94AF20E62DF72D0E94492431
:10469000A0910705B0910805EA0FFB1FE00FF11F7D
:1046A000E4910895EA81E350EA830895EA930E9431
:1046B0002D2385E08A95F1F70895E4E0E7BFE5E072
:1046C000EEBD0895EE27E7BFEEBD0895EA81FF270E
:1046D000E0930905F0930A05E881F981FA93EA93DA
:1046E0000C949C20FA93EA930E94D320EE27EA933D
:1046F0000C94AF20E3E0EA93E0EBF4E0FA93EA9362
:104700000C94DD20FA93EA93E8E1F0E0EBCFFA9322
:10471000EA93ECE0F0E0E6CFFA93EA93E6E0F0E02B
:10472000E1CFEE81FF27E0930905F0930A05EC81C4
:10473000FD81FA93EA930C949C20AA81BB81119786
:10474000AA83BB8311960895FA93EA93E8E0F0E018
:10475000C9CFFA93EA93E0E1F0E0C4CFEE81FF27FE
:10476000E0930905F0930A050895EC81FD81FA9321
:10477000EA930C949C20FA93EA93E0E3F0E0B2CF42
:10478000FA93EA930E942124E2E0EA930895E0EB91
:10479000F4E0FA93EA930C94DD20E3E0EA93E0EB93
:1047A000F4E0FA93EA930E940A21E2E0EA93EFCF61
:1047B000E4EFF1E0FA93EA930E942124E1E0EA9326
:1047C000E0EAF0E0FA93EA93E4E0F0E0FA93EA93A7
:1047D0000895FA93EA93E3E0F0E0FA93EA930895F8
:1047E0000E94F321E4EFF1E0CBCFE8ECF0E0FA93A4
:1047F000EA93E6E0F0E0FA93EA930895E2E0EA93C0
:10480000C6CFE4EFF1E0FA93EA930E942124E1E0BD
:10481000EA93EAEAF0E0FA93EA930895EE27EA933E
:10482000ECEDF0E0FA93EA930895E4EFF1E0FA9307
:10483000EA930C942124EA93E8EEF3E0FA93EA93E6
:104840000895E991F991309639F086E69EE0019756
:10485000F1F7A8953197C9F708950A921A92FA923A
:104860006A937A938A939A93AA93BA93EA93FA9360
:104870000FB60A92089509900FBEF991E991B99186
:10488000A9919991899179916991F99019900990DB
:104890000895EE0FFF1FEE0FFF1FEE0FFF1FEE0F2D
:1048A000FF1F0895EA17E1E009F0EE2708950024BC
:1048B0000A160B0608953A932A931A930A930895B9
:1048C0003B812A81198108810895FFFFFFFFFFFFC7
:1048D000FFFFFFFFFFFFFFFFFFFFFFFFFFFFFFFFE8
:1048E000FFFFFFFFFFFFFFFFFFFFFFFFFFFFFFFFD8
:1048F000FFFFFFFFFFFFFFFFFFFFFFFFFFFFFFFFC8
:10490000FFFFFFFFFFFFFFFFFFFFFFFFFFFFFFFFB7
:020000021000EC
:00000001FF
